S1230100BD0B917E0BA67E03CC7E03BD7E03477EE1D17EE1AC7E17257E03CC7E03BD7E03FF
S1230120477E03CC7E03BD7E03477E03E27E03D77E03527E03E27E03D77E03527E03E27E24
S123014003D77E03527E03E27E03D77E03521EE2010312180F5F037E13C57E13C57E13C5BF
S1230160524E4400176354414228001254494E542800172643485224280019024142532826
S123018000175B53474E2800174453515228001C2E4C4F4728001B2B45585028001BC35380
S12301A0494E28001AB6434F5328001AC64154414E28001C4B5045454B280017DC504F53DA
S12301C00017D654414E28001A6D56414C28001850415343280018274C454E280018414C3F
S12301E0454654242800187E524947485424280018DD4D4944242800189053545224280068
S12302001926464E0019CF555345522800171700BFFB4C495354000C5E4E4557000B99504C
S123022041544348000CAE474F535542000EC1474F544F000EE34F4E000EA25448454E00EB
S12302400E905052494E5400122D4C45540013B2494E505554000F90494600164D5245418D
S12302604400111F44415441001428524553544F524500119A454E44000BAB504F4B4528FD
S12302800017B952455455524E000F0C44494D001450444546001957464F520014F34E4591
S12302A058540015BD52454D00142354524143454F4E00141854524143454F464600141EED
S12302C04C494E453D0019124449474954533D00140653544F50000F20080013B252554E38
S12302E0000C28434F4E54000E314C4F4144000D0B53415645000CC7415050454E44000D54
S12303000E504F52543D0013F4544F00101F5354455000101F5245414459002044454C4556
S1230320544544001016FFFFFFFF0052452D454E544552004552524F522023200020494ED4
S1230340204C494E452000DE908613A7008611A70039DE906F016F036F006F026300863EB5
S1230360A701862EA70339A6008D0DA60008200C8DF58DF38620200E44444444840F8B30EC
S1230380813923028B0737368D17DF8ADE8CAD00DE8A323339DF8A37DE8EAD00DE8A3620DA
S12303A01137367E1ECB2B12DF8ACE8004BDE1ACDE8AB1015626037E0BAB323339DE90A693
S12303C0004724F9A601847F817F27F1DE90E600575724F8A70139DE90E6032AFAA602A72A
S12303E00239DE90817F2710A700C636E701C63EE701E6012AFCA60039CE031BBD045F208A
S123040008863FBD0386BD052ECE00B0BD03954D27FA810A27F6811527F2B1015327DA81B6
S12304200D2730B10154260EB60155BD03868C00B027D90920D67D008526038C00F82607B1
S12304406F00C6217E0BEBA7000820C08623BD038620B66F00DFAE96852603BD046E398D45
S123046006200BBD038608A600847F26F6398D15CE04788DF28D23390D0A15FFFFFFFF007F
S1230480FFFFFFFF00DF38DE3A0909DF3A369638A7009639A70132DE3839DE3AEE007C00DD
S12304A03B7C003B398DDEBD06500F9F2835DE3AEE0020148DCFBD06500F9F2835090909B5
S12304C009090909DF5DEE00C60532A700085A26F93232A7009E28010E8DBF398DA70F9F5E
S12304E02835200B8D9FBD06500F9F28AE0034C605DE5D32A700085A26F932A7016F009E32
S123050028010EBD06498D9239BD0370BD0485EE0009095CA60026FA0808085A5ABD0467B0
S12305208D0C7F0040BD049A0808087E045F368620BD12B33239BD0ABFBD062D251A16A6D1
S123054001BD062D2514BD0B13EE00AD00BD0649DE34313131310C390B39BD063A240781E3
S1230560242703098620080837E600C1282603088A8033BD0485DE2A9C460D2709E1002682
S12305800CA10126080CDF63BD049A0A396D012B1036A6018124322603BD065FBD0675208F
S12305A0D7EE0420D3BD03A17F00868D8928013936372541DF34DE634D2B1C0808DF63DEB2
S12305C05D9663A7009664A7018D7E3332812426029786DE340C39BD142E2405BD06852037
S12305E0015F37BD068517E601C1A42602D78633BD14B620C8DF34DE63E700A7014D2A191B
S1230600C60AE702E703BD142E25035FE703A602BD148E6D0327CA20C3A60181242605BD44
S1230620065F9786BD0675DF46DE63208E36847F81412B0F815A2F0E20093681302B0481DB
S1230640392F030D32390C3239DE5D8D29DF5D39DE5D8D0320F7090909090909090939373C
S1230660D63EC006DFAADBABD7ABC600D9AAD7AA33DEAA200808080808080808089C442B13
S1230680037E0E2C398D044D260C39BD04858DC0A60681052F05C6017E0BEB4F5F6D002B9F
S12306A0F56D062F215849D7529751584925E7584925E3DB52995125DDEB00890025D7BD30
S12306C008B16A0626DBBD049A39BD0ABFBD05A525097D00862627BD04E439BD102F2501ED
S12306E0398128261508BD078FBD0ABF812926020839C61301DF347E0BEBC60620F7C624B7
S123070020F38DC6BD0ABF815E27013908DF34DE5DBD0657E600372706BD1B2EBD0649DEFF
S123072034BD0ABF812D2608088D9FBD087D20028D98DF34DE5DBD0657A600335D26084D49
S12307402705BD06502022364D2A03BD087DBD0A3BBD1BC6324D2A0EBD0993BD1BA8BD062F
S123076049BD09C32003BD0649DE3420978D93BD0ABF812A260B08BD0ABF8D86BD0A3B2066
S1230780EE812F260908BD0702BD09C320E139BD0ABF7F0086812D2608088DD1BD087D20C8
S12307A007812B2601088DC5BD0ABF812B2608088DBBBD095C20F1812D2608088DAFBD0938
S12307C05920E54D39BD04858D497D00862605BD049A20BBBD0F7ABD049A8D379689817F2D
S12307E025037E18A0BD0ABF812B261E088D247D00862718BD0485BD0F7A09E601E70008BB
S12308005D26F8DF88BD049A20D24D39C624DF347E0BEBBD0ABF812226249786080F9F2840
S123082035DE88328122270BA700084D26F5C6047E0BEB6F0008DF88309E28010E39BD0ADA
S1230840BFBD05A52401397D00862725DF34BD0650EE000F9F2835DE88D63E32A7004D27DB
S123086006085A26F66F0008DF889E28010EDE3439BD065039BD0485BD0676200CBD0485B5
S1230880DE5D09092006BD0485BD06783637C6068699A000A700095A26F6BD06770DC6062F
S12308A08600A90019A700095A26F5BD049A333239368D08A600840FA70032393637DF5715
S12308C0C604DE57BD0678680086050969004A26FA5A26EE3332393637DF57A60084F097AB
S12308E053C604DE57640086050866004A26FA5A26F1DE57A6009B53A700333239BD048516
S1230900BD06507F0056BD13922419A6002A0B9756BD0886860FA400A700A60026088D9167
S12309206A0620F66F066F05A60681652D1537C6058699A700085A26FA8664A701BD065978
S12309403320D1819D2E03BD10E47D00562703BD0886BD0649BD049A39BD087DBD0485BD42
S12309600650BD13922428BD08D76C06BD0650BD13922411BD08D76C06A606A10D27082DF3
S1230980F38D1020EF8D0C8D23BD0649BD08FDBD049A39DE5D3736C607A60036A607A70064
S12309A032A707085A26F2DE5D3233393637DE5DC6060CA605A90C19A705095A26F5DE5DA2
S12309C0333239BD0485BD10E4BD0650BD13922505C6087E0BEB60068D38BD08D7BD08759C
S12309E0860B5F5C8DC66D002AF95ABD08758DBCBD0875BD0676BD0676BD08BCEB05E705DE
S1230A00DE5DBD08BC4A26DABD06498D867C00502059BD08D74F6D002A05BD08868680BDD3
S1230A2006506D002A05BD08868B80974AA606AB0D28058678240140975039BD0485BD066C
S1230A40508DCFDF59BD0649BD0993BD10E48609DE59E600BD08B15D2706BD09AC5A20F709
S1230A60DE5DBD0676BD08D74A26E5BD0650BD09939650A706BD0649BD08FD7D004A2A034C
S1230A80BD087DBD049A399632D633D03192302528DE2E9C2A27229630D631E001A200250B
S1230AA01A26035D2716DFAA4FE604DBAB99AAD7AB97AADEAA9C2A26DEDE2A0DDF2C39A6B6
S1230AC000812026030820F74D39BD102F2405C6077E0BEBDFACBD0650E60623F2C1042EAB
S1230AE0EE8605104D2706BD08D74A20F7A6019730A6029731DEAC0C39DE34A600084D2612
S1230B00FADF3639DE34A600084D2704813A26F6DF3639DFAC0F9F28CE015F2016DFAC0FCD
S1230B209F28CE0308200C8D96DFACDF340F9F28CE02119EAC340832812027FB815F2F02E1
S1230B4084DFE60027161127ED08BC015127178C020C271AE60026F1080820D7089FAC9FC1
S1230B60349E28010E399E28010ECE02DB397E101FFE014EDF2EDF2ADF464F9732973397C8
S1230B8040978697879754CE1725DF678620973E39BD1EB0B6015097968DD6864097928650
S1230BA03097937E0C28B6015097969E44CEA07FDF3A7F0085BD11B78613BD03868614BD4A
S1230BC00386BD046ECE0315BD045F7F0040BD044CCE00B0BD0ABFBD063A2505BD0D6A2008
S1230BE0EA4D27E7BD0B27EE006E009E44010101010ED720BD11B7BD046EDE5BEE00DF308C
S1230C00963426067F00307F0031CE0334BD0467CE0020BD0367CE033DBD0467CE0030BD48
S1230C200370BD046E7E0BABDE2EDF3CDF36CE0075DF65CE1E2FDF5FDE2ADF4686550908A5
S1230C408C8000270EA70001010101A10026046F0020EC09DF44DF947F00957E0E35BD111C
S1230C60BBCE0324BD045FDE34BD0ABF2729BD0ACADF34BD0A91DF24DE34BD0ABF270408EE
S1230C80BD0ACA4FC601DB3119D7319930199730BD0A91DE242006DE2ADF2CDE2E9C2C2745
S1230CA00A9C2A2706BD05090820F27E1428BD0AF9CE0E35DF20962136962036343434341B
S1230CC034BFA0087EE0E3BD11BB8612BD0386BD0D54BD0D54BD0D54BD0D5FBD0ABFBD0601
S1230CE02D250A168604BD038617BD0386DE2E9C2A270D8602BD0386BD0509088D5820EFB6
S1230D00B60156BD03868D577E0BABBD0B71BD11BB86119785BD0386BD0ABF16BD062D25F8
S1230D201737DE8EAD003381032603BD0395810426EFBD03951126E9BD0395810226F9BD50
S1230D400395BD063A25F4CE00B0BD040FCE00B08D1820E48D005F4F4A26FD5A26F939C64C
S1230D60328600BD03865A26F839BD0ACABD0A872411DEACBD0ABF271FDE2C9C2A271A8DB8
S1230D804E2015DEACBD0ABF260ADE2A9C2E27088D0F20048D0B8D37398D34DE30DF322036
S1230DA0F70F9F28DE2C9E2A08080808083434343434A60034084D26F99F2A9F4635DE2C29
S1230DC09C2A270632A7000820F69E28010E39DEACBD0B27DF48DE2ADF20D6AFD0ADCB069D
S1230DE037DB2B8600992A91442441D72B972ADE2ADF46330F9F2835DE209C2C270609A65F
S1230E00003620F6DE2C9630A700089631A700089648A700089649A70008E700089EAC3405
S1230E2032A700084D26F99E28010E39C6147E0BEBDE5BDF36CE1DB1DF5DDE94DF88DE36F2
S1230E409C2A26037E0BAB09A60008813A2605DF347E16967D003627EBDF5B7D0087272047
S1230E60BD0485BD11B7BD049A865BBD03868620BD0386BD0370865DBD0386BD046E20028B
S1230E800808080808DF34090909EE00EE006E00DE34BD0ABFBD063A24497E1696C6207E1E
S1230EA00BEBDE34BD078FBD06855D27F05AD755BD0B27EE008C0EE3272C8C0EC12705203D
S1230EC0DC7F0055DE36BD0B04DE658C00852605C6097E0BEB9636A700089637A70008DFE6
S1230EE06520037F0055BD03A1DE34BD0ACA7A00552B0ABD0ABF812C26A30820EEBD0A872A
S1230F002405C6077E0BEBDF367E0E35DE658C00752605C6107E0BEB0909DF65EE0020E789
S1230F20BD11B7CE02D2BD0467BD052EDE36BD0370BD0B04DF5B7E0BABBD0485C6FFD743CB
S1230F408D388D07BD049A397F0043DF88BD06500F9F28DE8835DE5DEE00D63E32A7007D60
S1230F6000432604812C27094D2706085A26ED20036F0034309E28010E3936DE889C94273D
S1230F800B099C94270609A60026F70832DF8839BD11BB96342605C6027E0BEBDE34BD0AA3
S1230FA0BF8122260DBD07C5812C26EB08DF34BD11A39696810A250A9785BD04097F0085F5
S1230FC02003BD0401CE00B0DFACDE34BD13AB2440DF34DEAC7D008626158D48241C4D27CA
S1230FE006CE032BBD045FBD0401CE00B020E6BD0ABF010101BD0F482003BD04B4BD0ABFCA
S1231000812C260108DFACDE34BD0ABF08812C27BB097F0040813A27034D26037E1428C693
S1231020037E0BEBBD0ABF974A08812D2704097F004A4F974C974D974EBD10E4D65DD7263F
S1231040D65ED727C605BD0ABFBD063A240B812E2605974D0820EF0D390908A600BD063A0E
S123106025428030260F7D004C260C7D004D27EA7A004B20E5974CBD0485DE265D27167D3C
S1231080004E2608AB00A700085A200648484848A70073004EDF267D004D26037C004BBDF2
S12310A0049A20B67D004D2608812E2604974D20A95F8145261408A600812D2709812B267D
S12310C001088D362004088D3150964B1BBD0485DE5DA706BD0649BD049A7D004A2703BDC7
S12310E0087D0C39BD048537C607DE5D6F00085A26FA7F004B33BD049A39A600BD063A2454
S123110005C6027E0BEB80301608A600BD063A250D581758581B16A60080301B160839DEF1
S123112034BD13AB2469DF34DE3C9C2E273E7D00862720BD0ABF272A81222705BD0F4820EF
S12311403BDF3CDE94DF88DE3CBD0813250ABD0F392029BD1024242101A6002705C6197E87
S12311600BEB9C2A27F7A600084D26F6A603816926F0080808080820B5BD04B4A600812C0C
S1231180260108DF3CDE34BD0ABF08812C279209813A27034D26C67E1428DE2EDF3CDE34E1
S12311A07E1428BD0485BD0F7AA6002706BD12B30820F6BD049A3996962025DE34BD0ABFD5
S12311C0812326F308BD078F2710812C270B813B2707813A27047E13C508DF34BD0685173D
S12311E08108250C7F009097918609164848201016484891912601393697918680979032B0
S1231200481BCE0106DF8CDF8E9B8D978D8B03978F9690270DDE90A60381FF2605C6267E34
S12312200BEBDE8E0808080FAD00010E398D8CDE34BD0ABF813A27034D263109A6000881BA
S12312403B2706BD046E7F004008DF367E0E357E0BEB0101BD17B1BD049EBD06855AD0404A
S12312602F06BD052E5A26FA9E44200FBD07C57D008626048D642003BD11A3BD0ABF812C4C
S1231280260E08964016C4F010270ABD052E20F3813B260B0896902698862C8D1620924DFD
S12312A0278F813A278BC60620A5862E20054F840F8B3036BD038632812024013937D64006
S12312C05C7D00922710D193250CD192240481202604BD046E5FD7403339BD0485965497A5
S12312E0A9BD06504F974D6D00260D7D00A926208DBCBD049A7E052E6D002A07862D8DB309
S1231300BD0886A60681092E3C81FF2D384D2E158D9C8D96974D6D062A278D927A00A9270C
S1231320D16C0620F17D004D2617A6008D81BD08B16A0626F57D00A926048D5624B4BD12BF
S1231340AA8D3620ADA600BD12AFBD08B1BD12AA8D278645BD12B3E606813A27035A2A06E0
S1231360862DBD12B3504F4CC00A2AFB4ACB0ABD12AF17BD12AF7E12F2D6A98D15240DA6AE
S123138000BD12AFBD08B15A26F120057D005426EE39BD0485DE5D37C6066D002607085A21
S12313A026F80C20010DBD049A3339BD05A525080D39DE348DF52505C6127E0BEBBD0ABFA0
S12313C008813D2704C60620F17D0086260FBD078F813A27034D26EDBD04B4204BBD07C502
S12313E07D008626037E080C813A27034D26D6BD0F392034DE34BD078FBD068517BD11E032
S1231400DE34D7962022DE34BD078FBD0685C10A2502C609D754201086FF9787200A7F00F2
S1231420872005BD0AF92003BD0B047E0E35BD0485DE34BD078F08812C270B8129261DDF2E
S123144034BD049A0C39BD06E6DF34BD049A0D39DE347F0086BD053629022505C6057E0B9F
S1231460EB4D2AF8DF34DE63E700A7018DC02405BD068520015FE703BD068517A7028D0E60
S1231480DE34BD0ABF08812C27C8097E1428BD0485E601C1A42602D786E6038D197D0086A0
S12314A02703BD065FBD0677DF46BD049A9646A7049647A705394D2605C6157E0BEBA1026F
S12314C022F7E10322F336A60297515D27155A27129651BD06777D00862703BD065F4A2624
S12314E0F220EB32BD06777D00862703BD065F4A26F239DE34BD13AB25037E13B87D008694
S123150026F8DF34BD0B04DE5DBD0657A600E6019751D752CE1E2F9651D6529C5F271CA1CE
S1231520002610E101260C9636D637A10E2604E10F2708BD0675BD067520DC8C1EAF26059C
S1231540C6167E0BEB9651D652A70008E70008DF5FDE34BD0ABF08813D27037E13C5BD07AA
S12315608FBD04B4BD0B1D8C030C26EFDE34BD078FDF34DE5FBD04A5BD0677DF5FDE34BD6C
S12315800B1D8C03132609DE34BD078FDF342003BD1BA8DE5FBD04A5BD0677DF5FDE34BD49
S12315A00ABF813A27034D26B208DF36DE5FD636E70008D637E70008DF5F7E0E35DE34BD35
S12315C013AB25037E13B8BD0ABF813A27034D26D608DF36BD0650A600E601DE5F8C1E2F51
S12315E02766DF5F8C1E2F275BBD0656BD0656A10026EFE10126EBDF61EE00BD04DCDE61DC
S1231600BD067586026D002A028B03974FBD04DCBD095CCE006FBD04A5BD0649DE6108083C
S1231620BD04DCBD16DB2407DE61DF5F7E0E35CE006FBD04DCDE61EE00BD04A5DE61EE0E4A
S1231640DF3620E8C6182002C6177E0BEBDE34BD07C58D4B974F7D0086272FBD07C57D0060
S12316608626037E080CDF34BD0F7ADF20BD0F7A0F9F2835DE20324D2707A00026050820DE
S1231680F5A6009E280E8D5B2007BD078FDF348D4A24037E1423DE34BD0B27EE006E00BD95
S12316A00ABF08813D2603860039E600813C2613C13D260408860239C13E260408860339EF
S12316C0860139813E2705C6067E0BEBC13D260408860539C13C27E4860439BD0959BD067A
S12316E050A60036964F4848CE16FDDF209B21972186009920972032DE204D6E00271620B3
S1231700122B12200E2B0E20F4260A200627042B022A020D390C39BD17ABBD0485DE67ADDF
S1231720000FBD049A39BD17ABC609E0065D2F08BD08D76C065A20F56F05BD0649BD08FD7B
S1231740BD0650398D65A6002710974ABD1BA8BD06507D004A2A03BD0886398D4E6D002A0C
S1231760F920F4DE34BD0ABF8128260F08DF348D3ABD13922405BD06492008CE00696C009E
S1231780BD04DCCE1CC7BD04DCBD0A3BBD0650BD08B1A60136A603A70132A7036F06BD068D
S12317A049BD08FDCE0069BD04A5398D04BD065039DE34BD06E6DF3439BD142E25037E06B5
S12317C0F2BD068537BD068BD7529751DE5133E700DE347E142896404C8D11398DD3BD0604
S12317E08BD7529751DE51A6008D0139BD0485DE5DBD10E4C609E7065F80645C24FB5A8B1C
S123180064E704BD08BC5F800A5C24FB5A8B0AEB04E704BD08BCAB04A704BD0649BD08FD1E
S1231820BD0650BD049A398D47A60008812927037E06F2DF34BD0F7AA600BD17EC7F00866D
S1231840398DE44F4CE600085D26F94ABD17EC398DD5BD10242405C6277E0BEBBD06503969
S12318608D0EBD0ABF812C27037E06FA08DF3439DE34BD07C57D008626037E080C398DE09B
S1231880BD06E6DF34BD06855C37C180241220208DCEBD142EC67F2403BD0685C18025057D
S12318A0C6257E0BEB5C37BD0685C18024F2174ABD0F7A084A2AFC09324A0F9F2835DE887E
S12318C04D2B0833E700084A5D26F5096F00089E28010EDF88C6FFD786BD0650398D81BDAB
S12318E006E6DF34BD0685C18024B5BD0F7A37E600084C5D26F94A3336102A014F16DE8897
S123190020B1BD17B1BD0685DE88E700086F000820C1DE34BD078FBD0685D792175757108D
S12319204C97937E1428BD142E24037E080CDE8CBD0485964036CE194FDF8CBD12DA3297EC
S123194040BD049ADF8CDE88096F00087E18D3DE88A70008DF8839DE34BD0ABF276C814687
S1231960266808A600814E266108A600BD062D2559BD0AC581282652BD0AC52A037E142895
S12319808A80A700BD05362941C47FD7529751DF34DE63E700DE34BD0ABF8129262CBD0A46
S12319A0C5813D262508E600C13A271A5D2717D15226F2A601BD063A24028620915126E5F8
S12319C0CA80E70020DF097E1428C6227E0BEBDE34E600BD0AC58128264E08BD0485DE2EB9
S12319E09C2A2744080808A6000881962705BD0AFB20EDBD0AC50808A6001126F1BD0AC5E4
S1231A0008BD05A52522BD0AC5BD0AC5DF24BD049ABD06E6BD04B4BD0485DE24BD078FBD20
S1231A200650BD049ADF3439C6237E0BEBBD17B18D66CE1CD9BD04DCBD09C3BD0650BD1700
S1231A4029BD0649CE1CD9BD04DCBD0A3BBD0959BD1A98CE1CD3BD04DCBD0959BD06506D64
S1231A60002B09CE1CD9BD04DCBD0959398D47BD06498D5A6D0026088601A700869AA70619
S1231A80BD0649BD09C3BD1B0B398D0C8D0ABD0A3BCE0097BD04A539DE5DBD0657A600A7B9
S1231AA007089C5D26F77E0649CE009DBD04A5BD10E4BD064939BD1A2D8DCF8DECC607CEF5
S1231AC01D458D222045BD1A2D8DBFBD0650BD1BA88DD6C607CE1D6F8D0C8D2FA60681FAA3
S1231AE02C03BD10E439DF4137CE0097BD04DCBD0A3BDE41BD04DCBD0658BD095C335A26C2
S1231B00E5CE009DBD04DCBD0A3B39BD10E4DE5DBD0657E606E70D6D00270AC650E70BBD50
S1231B200649BD095CBD06506F0439BD17B1BD10E4DE5DBD0657A606C601E706D74EE6007B
S1231B402F61C10325056F067F004EBD0649CE1CE5914E27182A0B36BD04DCBD0959324C23
S1231B6020EC36BD04DCBD095C324A20E1CE00A3BD04A58D33BD0959BD1A988D3ABD095CD5
S1231B80BD09C3BD1A8ABD1AA9C609CE1D1BBD1AE68D24BD0A3BCE00A3BD04DCBD095CBDA5
S1231BA0065039C6287E0BEBDE5DBD10E48601A700A706BD064939DE5DBD10E48602A70009
S1231BC04A20EEBD17B1BD1A98CE1CE5BD04DCBD09C3BD0650BD1729E600BD0649BD1A984F
S1231BE05D2A09BD087DBD0685502003BD068537CE1CE5BD04DCBD0A3BBD0959CE1CDFBDC2
S1231C0004DCBD0A3BCE0097BD04A5BD1BA8BD1AA9C60ACE1DABBD1AE6BD1A98BD0A3BBDC2
S1231C201A98BD0A3BBD1B0B33EB06E70639BD17AB6D00260139BD0649BD1B2EBD0649CE87
S1231C401D81BD04DCBD0A3B7E1BC6BD17B1BD1BA8BD0650BD0650A600362A03BD08867FE6
S1231C600043A6062F059743BD0993BD0649BD0649BD09C3BD1A8ABD1AA9C607CE1CC1BD53
S1231C801AE67D0043270CBD087DCE1CCDBD04DCBD095C324D2A03BD087D7E1B0B099999C8
S1231CA06100009666826200000198078700009867664900000796263200FF966393730017
S1231CC0FF0681241100FE08372541690001570796320103141592650106283185300102D6
S1231CE0500000000002302585100101000000000103333333330002000000000001428508
S1231D007143000111111111000909090909FF0769230769FF0666666667FF058823529464
S1231D20FF0100000000019833333333000833333333FE9801587302FD0275573192FB97E2
S1231D4049478916F90160590438F70100000000019500000000000416666667FF9861117D
S1231D601111FE0248015873FC9724426808FA0208767570F8010000000001010000000066
S1231D80010500000000000166666667000416666667FF0833333333FE0138888889FE01B0
S1231DA098412698FD0248015873FC0275573192FB2EDD700000000304000000000001006A
S1231DC008700000000308ED3F019C0000FD8D7519458CE0C2DF3A0920681DDC9041DD498E
S1231DE0213D01FF0F001108B95F1B258C2C0169FD84914900FD80EFFB4101DD016319057C
S1231E0091A0488EA0478D498D3C815826FA8D3681312707813926F07EE1157F1E008D2601
S1231E20165C8D22B71E018D1DB71E02FE1E018D15A70001A100260B085A26F38D087C1E43
S1231E400027C57EE0408D1436BB1E00B71E0032398611BDE1D1863CB780073937BDE1A54B
S1231E60A6002BFC6F02BDE1F3BDE1EFC604E70258BDE1EF0D6900465A26F6BDE1EF7EE14C
S1231E80E300443FEF47FF06FEFF64F7FF1A5F0662D76EB3F602AF9FEFF36F8246BF24F734
S1231EA0FF00FF00F0F6EFDEAEB26F9FE686FF007F00917DE0D62B0FBDE1D32607FEA010CB
S1231EC07F1EAF39FEA0107A1EAF397D1EAF260CB680044724037E03A87E03BAB680047E0B
S1231EE003A60027DE267D00252621F01B83B21B822503FF1B82B61B80F61B81D0279226EE
S1041F0025B7
S105A048010011
S9030000FC
